:020000021000EC
:10F8000011241FBECFEFD1E4DEBFCDBF12E0A0E0D8
:10F81000B2E0EEE4FCEF01E00BBF02C007900D92F6
:10F82000A030B107D9F713E0A0E0B2E001C01D920B
:10F83000A030B107E1F70E9446FC0C9425FE0C9421
:10F8400045FC9091C00095FFFCCF8093C6000895C1
:10F850008091C00087FFFCCF8091C600089581E4AD
:10F860000E9421FC86E50E9421FC82E50E9421FC89
:10F8700082E40E9421FC8FE40E9421FC8FE40E941C
:10F8800021FC84E50E9421FC08950895CF93DF9325
:10F89000CDB7DEB728970FB6F894DEBF0FBECDBF49
:10F8A000F89498E10FB6F89490936000109260007D
:10F8B0000FBE84B7877F84BF80916000886180938A
:10F8C00060001092600080E88093610010926100F7
:10F8D0006C9A749889E18093C4001092C50082E00C
:10F8E0008093C0009093C10086E88093C200CC242E
:10F8F000DD24EE24FF2400E21EE48091C00087FF97
:10F9000004C08091C600833579F02CE2C21621E054
:10F91000D20618F04798F7010995C8010197F1F749
:10F920000894C11CD11CE9CF0E942FFC9924CC243F
:10F93000DD2490E1692E8824839423E0522E31E166
:10F94000732E8EB186258EB90E9428FC813611F463
:10F9500089E562C1813469F40E9428FC8A83198296
:10F960000E9428FCC82EDD2489819A81C82AD92AC0
:10F9700037C1823629F489E50E9421FC81E020C14B
:10F98000823409F08AC00E9428FC8C831B820E946A
:10F9900028FC082F10E0AB81BC810A2B1B2B0E9496
:10F9A00028FC982F80E0E82E82E0F82EAA24BB24C1
:10F9B000A016B10628F49F830E9428FC9F8101C0F5
:10F9C0008FEFF70181937F010894A11CB11CF0E037
:10F9D000AF16F1E0BF0661F724E4921609F0F2C019
:10F9E000963409F03CC0EE24FF24CC0CDD1CEE1C48
:10F9F000FF1C80910002A0E0B2E0B701A60190E0F8
:10FA000011963C9011972224822993290C01FA0126
:10FA100060935B0080925700E89511244E5F5F4F22
:10FA20006F4F7F4F0250104029F012968C91129721
:10FA30001296E5CF85E0F601E0925B0080935700D7
:10FA4000E89507B600FCFDCF70925700E895DB0102
:10FA5000CA01B695A795979587956C01C1C0953455
:10FA600009F0BEC09801760140E0A42E42E0B42E19
:10FA7000D5016D915D01C7012F8338870E9417FE64
:10FA80000894E11CF11C2F8138852150304081F70A
:10FA9000C00ED11EF999FECFA3C0873609F056C01B
:10FAA0000E9428FC8E831D820E9428FC082F10E0F3
:10FAB000ED81FE810E2B1F2B0E9428FC863481F5E0
:10FAC000EE24FF24CC0CDD1CEE1CFF1CFFEFCF1638
:10FAD000F7EFDF06F1E0EF06F0E0FF0628F4EBBEFB
:10FAE000F601A790B69003C0AA24AA94BA2C8A2D36
:10FAF0000E9421FC8B2D0E9421FC82E090E0A0E07E
:10FB0000B0E0C80ED91EEA1EFB1E02501040F1F6EE
:10FB1000D701C601B695A795979587956C0111CF2A
:10FB2000853409F00ECF58017601C7010E940FFEFF
:10FB30000E9421FC0894E11CF11C0894A108B10862
:10FB4000A114B10491F7C00ED11EFBCE853609F584
:10FB500094E4991609F044C080E090E0A0E0B0E0A1
:10FB6000FC01A0935B0050925700E89507B600FC9B
:10FB7000FDCF80509F4FAF4FBF4F8030E8EF9E07C3
:10FB8000E1E0AE07E0E0BE0759F770925700E89554
:10FB900027C0853451F48DE00E9421FC85BE15BE3E
:10FBA000749AE0E0F0E00995CCCE8035C9F08C3451
:10FBB000B9F0803711F483E52FC0843729F484E449
:10FBC0000E9421FC80E028C0982F9857923018F4AA
:10FBD0000E9428FC05C0843529F40E9428FC982E38
:10FBE0008DE01AC0833519F40E942FFCAACE863509
:10FBF00029F480E30E9421FC88E30EC0833741F49E
:10FC000081E00E9421FC87EA0E9421FC8EE104C071
:10FC10008B3109F496CE8FE30E9421FC92CEF999A4
:10FC2000FECF92BD81BDF89A992780B50895262F01
:10FC3000F999FECF1FBA92BD81BD20BD0FB6F894D1
:0EFC4000FA9AF99A0FBE01960895F894FFCF34
:040000031000F800F1
:00000001FF
